:020000040000FA
:10000000831685108511FF30860083128F019C01B5
:100010009C1485101030840085118001061E801408
:100020000000840A00008001000000000000840A33
:1000300000008001000000000000840A851180019A
:10004000861E80140000840A00008001061C8014B3
:100050000000840A00008001861C80140000840ACD
:1000600085158001061D80140000840A8515800115
:10007000861D80140000840A85158001061E8014E8
:100080000000840A85158001861E80140000840A01
:1000900000008001000000000000840A00008001D0
:1000A000000000000000840A0F3084000E308E0033
:1000B0000508FD3900040418023A8500840A4E3010
:1000C000722000008E0B58288510FF307220FF3000
:1000D0007220FF307220FF3072206F3072200000DB
:0C00E00064000A288C008C0B73280800B8
:02400E00FE3F73
:00000001FF
